:1000000007308A00332F0000633479316100C43235
:100010006E1DA0126C320D050000413DE936753AA7
:100020003A102536E4060A004536653BE3323A10BD
:1000300025320D0500105A08F8015902031823282B
:100040005908F7002F28F7010830DB00D90DF70D0C
:100050005A0877020318F700F80DDB0B2628080072
:100060008E30F70083164B08F8004A08F900FA01B1
:10007000F808031D45287908F800F9010830F7024F
:10008000F808031D4528F7014D280310F81B4C28DC
:10009000F90DF80DF7034528F81383120800A01393
:1000A000200883168700831287130830F800582829
:1000B0000000F8176928F813E50C03188717031CCC
:1000C0008713781769287813F80B5C2867280000D5
:1000D00087173F308400840B6B280000F81B5B28D7
:1000E000781B63280800831603178C170C14000074
:1000F00000000318A22883120C087F390313DD00C7
:1001000003170D080313DE0003170F080313DF00A6
:100110005D08E5004F205E0803178D0003135F089C
:1001200003178F0083168C170C1400000000831235
:100130000313DC0B9C289F2883160317A228C128D1
:100140008316031783120C0D0E0D7F390313DD0088
:1001500003170D080313DE0003170F080313DF0056
:100160005D08E5004F205E0803178D0003135F084C
:1001700003178F008D0A03198F0A03100313DC0B7A
:1001800073280800E4010408E3006410831B64146E
:10019000DD1FD228E317631EE30ADC09DD09DC0A50
:1001A0000319DD0A5D0EF038DF00DF07E23EE000F4
:1001B000323EE2005D080F39E007E007E207E93E62
:1001C000E100E107E1075C0E0F39E107E207E10D0D
:1001D000E20DE209E20D5C080F39E207DF0D07309E
:1001E000DE000A30E207E103031CF228E107E00326
:1001F000031CF628E007DF03031CFA28DF07DE03F1
:10020000031CFE285E3084008313073063056313EC
:1002100084036305031D1329631A840A631A1329CF
:100220002030F70030298407623004020319631775
:100230000008F700031D2429631B2429631A3E29A3
:10024000E319242920302F29E31F2C292D30F70012
:1002500084036313E3133029E31563123030F70787
:10026000DD010408DC005D10831B5D147708E500E8
:100270004F205C08840083135D188317840A631F72
:1002800014290800831646080319082AD2004A08D0
:100290000319082AD202031C52297F30D2070318FF
:1002A000082A58298130D202031C082A0319082A77
:1002B0005208F700F801F901FA01D1014708D0000E
:1002C000D0174808CF004908CE001930D2004D0899
:1002D000CE0203187B290130CF0203187B29D002FC
:1002E00003187B29D10203187B29D10AD00ACF0A2F
:1002F0004D08CE07AD294C08CF02031896290130CE
:10030000D00203189629D10203189629D10AD00ADF
:100310004C08CF074D08CE07031CAD29CF0A031D9B
:10032000AD29D00A031DAD29D10AAD294B0880386B
:10033000D0020318AC290130D1020318AC29D10A2C
:100340004B088038D0074C08CF07031C8A29D00AF5
:10035000031D8A29D10A8A297A14D20BB029BB2914
:100360000310CE0DCF0DD00DD10D0310FA0DF90DE8
:10037000F80DD30D6729531CC3290310F80CF90C91
:10038000FA0CD30CC629F7030319082AD31BEF294B
:100390000310CE0DCF0DD00DD10D4D08CE02031898
:1003A000DB290130CF020318DB29D0020318DB2937
:1003B000D102031CFE294C08CF020318E6290130A4
:1003C000D0020318E629D102031CFE294B0880380D
:1003D000D0020318EF290130D102031CFE29FA0ACA
:1003E000031DFE29F90A031DFE29F80A031DFE2933
:1003F000F70A0319082AF80CF90CFA0C4708D2007E
:100400004B08D206D21F062AF8170C2AF8130C2A1A
:10041000F701F801F901FA018312080083164A086E
:1004200003197F2AD2004E0803197F2AD207031826
:10043000202A7F30D202031C7F2A03197F2A242A14
:100440008130D20703187F2A5208F700F801F9011A
:10045000FA014B08D600D6174C08D5004D08D40039
:100460001830D200D301541C4D2A5108FA07031C3E
:100470003F2AF90A031D3F2AF80A0319D317500827
:10048000F907031C462AF80A0319D3174F08CC00B2
:10049000CC174C08F8070318D317D30DF80CF90C38
:1004A000FA0CD60CD50CD40C0310D20B322A013026
:1004B000F70703187F2AF81B642AD60DFA0DF90DE9
:1004C000F80DF70303197F2AD61F752AFA0A031DB0
:1004D000752AF90A031D752AF80A031D752AF80CF6
:1004E000F90CFA0CF70A03197F2A4B08D3004F08BE
:1004F000D306D31F7D2AF817832AF813832AF7011E
:10050000F801F901FA01831208006E088316C90088
:1005100083126D088316C80083126C088316C70007
:1005200083126B088316C600CD01CC013430CB009A
:100530008630CA00831242217708F3007808F4005D
:100540007908F5007A08F6008316CD007908CC000A
:100550007808CB007708CA00C330D100F530D0004E
:100560004830CF008030CE0083120E227A08F2008D
:100570007908F1007808F0007708EF006F08F700BD
:100580007008F8007108F9007208FA00080080305D
:10059000831CCD2A8316CF0683128316D401D5017E
:1005A0004B08D3004F08D3064A080319BB2BD200CF
:1005B000F7004E080319C42BD2020319602B031C49
:1005C0001E2B4F08D800D8175008D7005108D60066
:1005D000D5010310D80CD70CD60CD50CD20BE82AB9
:1005E000D31FF52A5414D82B541052105416CD3062
:1005F00084008313ED2B5412D31B082B521C132B96
:10060000D80CD70CD60CD50CF70A0319D32B132B07
:10061000D81B162B0310D50DD60DD70DD80DF7030B
:100620000319D32B082B5417802B54134B08D300DA
:10063000D31F1C2BD817CC2BD813CC2B4E08D20091
:10064000F7004A08D2024B08D800D8174C08D70048
:100650004D08D600D5010310D80CD70CD60CD50CFC
:10066000D20B2A2BD31F372BD414D82BD4105210D3
:10067000D416D13084008313ED2BD412D31B4A2B14
:10068000521C552BD80CD70CD60CD50CF70A0319D5
:10069000D32B552BD81B582B0310D50DD60DD70DAA
:1006A000D80DF7030319D32B4A2BD417802BD4135F
:1006B0004F08D300D31F5E2BD817CC2BD813CC2BCD
:1006C0004F08D800D8175008D7005108D600D31FBC
:1006D0006D2BD8135415D82B5411D5015210CD3091
:1006E00084008313ED2BD31B962B4B08D300521C95
:1006F000802BD80CD70CD60CD50CF70A0319D32BAA
:10070000D51F912BD60A031D912BD70A031D912BC0
:10071000D80A031D912BD80CD70CD60CF70A031955
:10072000D32B541B152BD41B572BB52B8030D8063D
:10073000D81F9E2BD82B4F08D300AB2B4B08D300D0
:10074000D808031DAB2BD708031DAB2BD608031D00
:10075000AB2BF701CC2BD81BB52B0310D50DD60D29
:10076000D70DD80DF70BAB2BD32BD31FB92BD81725
:10077000CC2BD813CC2B4E08F7004F08D8005008CC
:10078000D7005108D600CC2B4A08F7004B08D800F8
:100790004C08D7004D08D6005808F8005708F90053
:1007A0005608FA000B2CF701F801F901FA010B2C9D
:1007B000D501D609D709D809D509D50A031DE62BD5
:1007C000D60A031DE62BD70A0319D80A5418F42AAF
:1007D000D418362B54196C2B9B2B0008D607031CFE
:1007E000F72BD70A031DF72BD80A031952148403D9
:1007F0000008D707031CFF2BD80A031952148403DF
:100800000008801F803AD80703185214541AFB2A94
:10081000D41A3D2B732B8312080083164708CE0091
:100820004B08CE06CE1F192C03110310C71B03144F
:100830004C2C4708CE004A08CF004608CF020319C7
:10084000272CCE1F4C2C0308013A83004C2C4B085C
:10085000CF004708CF020319332CCE1F4C2C0308BE
:10086000013A83004C2C4C08CF004808CF020319F2
:100870003F2CCE1F4C2C0308013A83004C2C4D0812
:10088000CF004908CF0203194B2CCE1F4C2C030874
:10089000013A83004C2C0310831208008E30F700BD
:1008A00083164608F7024708F9004808F800F917C8
:1008B000F7080319662C0310F908031D622CF808C9
:1008C0000319662CF90CF80CF70B5B2CC71F6D2C69
:1008D000F809F909F80A0319F90A831208008316BE
:1008E000A701A601A5017F30A4007E30AE008030B4
:1008F000AF00B001B1017A30B2002A30B300AA30A3
:10090000B400AB30B5007530B600B630B7000B3070
:10091000B8006130B9006F30BA005030BB000D3004
:10092000BC000130BD006930BE009330BF00F23022
:10093000C0007E30C1006230C2000F30C30076308C
:10094000C400AE30C5007608C9007508C800740838
:10095000C7007308C600CD01CC01CB01CA018312C8
:100960000D24031CB62C7408803AF4007608831614
:10097000C9007508C8007408C7007308C600DB30DA
:10098000CD000F30CC004930CB007F30CA0083123D
:1009900042217A088316C9007908C8007808C70080
:1009A0007708C60083124E2478088316A8007608BC
:1009B000C9007508C8007408C7007308C600DB309A
:1009C000CD000F30CC004930CB007F30CA008312FD
:1009D000422177088316C6007808C7007908C80046
:1009E0007A08C900CB012808CA008312302083147A
:1009F00083164908CD004808CC004708CB004608BC
:100A0000CA007A08D1007908D0007808CF007708AA
:100A1000CE008312C7227A088316AD007908AC0095
:100A20007808AB007708AA000330A805A8080319C6
:100A30001D2D2808023C031D392D2D08CD002C0842
:100A4000CC002B08CB002A08CA00DB30D1000F30C5
:100A5000D0004930CF007F30CE0083120E227A08BA
:100A60008316A3007908A2007808A1007708A000E7
:100A7000A22D280B6F2D8314CD01CC01CB017F302B
:100A8000CA002D08D1002C08D0002B08CF002A085E
:100A9000CE008312C72277088316C6007808C700E5
:100AA0007908C8007A08C900CD004808CC0047087A
:100AB000CB004608CA00DB30D1000F30D0004930EF
:100AC000CF007F30CE0083120E227A088316A30057
:100AD0007908A2007808A1007708A000A22D83144D
:100AE0002D08CD002C08CC002B08CB002A08CA000A
:100AF000D101D001CF017F30CE008312C722770809
:100B00008316C6007808C7007908C8007A08C900AB
:100B1000CD004808CC004708CB004608CA00DB30AF
:100B2000D1000F30D0004930CF007F30CE0083128B
:100B30000E227A088316A3007908A2007808A10083
:100B40007708A000FE01FD01FC017F30FB002308B7
:100B5000CD002208CC002108CB002008CA002308C1
:100B6000D1002208D0002108CF002008CE00831237
:100B70000E227A088316A3007908A2007808A10043
:100B80007708A000A9012908053C031C312E27087D
:100B9000CD002608CC002508CB002408CA00230875
:100BA000D1002208D0002108CF002008CE008312F7
:100BB0000E227A088316A7007908A6007808A500F7
:100BC0007708A400290DF700F70DFC30F70577082A
:100BD000AE3E840083130008C600840A0008C700E4
:100BE000840A0008C800840A0008C900CD0048082B
:100BF000CC004708CB004608CA002708D1002608C9
:100C0000D0002508CF002408CE0083120E228316C0
:100C1000C7010408C6004710831B471483107E08D1
:100C2000CD007D08CC007C08CB007B08CA007A0888
:100C3000D1007908D0007808CF007708CE00831261
:100C4000C7228316460884008313471883177A083F
:100C5000FE007908FD007808FC007708FB00A90A6F
:100C6000C32D2808023C0319372E280B3A2E7C0886
:100C7000803AFC007B08F7007C08F8007D08F9004A
:100C80007E08FA008312080083146E088316CD00D4
:100C900083126D088316CC0083126C088316CB0078
:100CA00083126B088316CA00DB30D1000F30D000EE
:100CB0004930CF007F30CE008312C7227708EF0083
:100CC0007808F0007908F1007A08F200F600790857
:100CD000F5007808F4007708F3006F2408005C083A
:100CE0008316C90083125B088316C80083125A0852
:100CF0008316C700831259088316C600C330CD007F
:100D0000F530CC004830CB008030CA00831242213D
:100D10007708DE007808DF007908E0007A08E10053
:100D20008316CD00831260088316CC0083125F08FF
:100D30008316CB0083125E088316CA00D101D0014E
:100D40003430CF008630CE0083120E227A0883160C
:100D5000C9007908C8007808C7007708C600831260
:100D60004E247808DD005D08F80008002030251EBC
:100D70003030A6002408F700A41FC52EF709F70A93
:100D80007708A4002D30A600A5172408D9006430E8
:100D9000DA001B207708A40030307807A700240869
:100DA000D9000A30DA001B2030307707A900303034
:100DB0007807A8002608F700A51DE02EA51F25111D
:100DC000251AED2EA51F082F2519082F7708A70033
:100DD000A518082F7708A800082F30302702031D18
:100DE000082F7708A7002030A600A51DFB2E25118F
:100DF000A514A51FA51030302802031D082F770861
:100E0000A8002030A700A51DFB2EA510A51F2510AA
:100E1000251D0D2F2608E5004F20A51C122F2708A1
:100E2000E5004F20251C172F2808E5004F20290832
:100E3000E5004F208A110A12D72F25308400831332
:100E400000080319302F0230F800F701F70B262FA6
:100E5000F80B252F9730F700F70B2C2F800B232F43
:100E60008A110A12E22F840183131F308305713027
:100E700083168F000F088312A013200883168700A3
:100E800083128717831603170908C03989000313D3
:100E90001F129F12003003178800831287018801F8
:100EA0008901FF300313A000831603170908C03916
:100EB000890003131F129F1200300317880083124A
:100EC00003131F139F1383169F1383121F1494126F
:100ED000A01220088316870083122016200883168C
:100EE00087008312A0112008831687000130831227
:100EF00094000030831694000108C7390838810037
:100F0000831290010030F8009200003083169200A6
:100F100083122015200883168700831297018316F9
:100F20009B019C0101309D008312031787018801FA
:100F300089010B300313A4001230A5000E30A60067
:100F4000A701A801AC01AB014430AA008430A9007C
:100F5000B001AF016030AE008230AD000A1600284B
:100F60000A120D3003178D0000308F000310083077
:100F70000313DC007320103084002208DD002108F8
:100F8000DC00C2200D30E5004F200A30E5004F2084
:100F9000143003178D0000308F0003100830031346
:100FA000DC0073202308A4001F30A500B62E0D30EE
:100FB000E5004F200A30E5004F200830A400FA3049
:0E0FC000A5001D2FA40BDF2F0317992F630030
:1010000074106A08EF006908EE006808ED006708D0
:10101000EC006A088316C900831269088316C800A9
:10102000831268088316C700831267088316C600F8
:10103000CD01CC01CB01CA018A1183120D248A157E
:10104000031C262874146D08803AED008316C9012C
:10105000C801C7017E30C60083126F088316CD0019
:1010600083126E088316CC0083126D088316CB00A2
:1010700083126C088316CA008A1183120D248A1504
:10108000031C332983148316CD01CC01CB017F309F
:10109000CA0083126F088316D10083126E0883166C
:1010A000D00083126D088316CF0083126C0883165C
:1010B000CE008A118312C7228A1577088316A400EE
:1010C0007808A5007908A6007A08A7002708C900B3
:1010D0002608C8002508C7002408C600CD01CC0199
:1010E000CB018030CA008A11831242218A15770809
:1010F0008316A4007808A5007908A6007A08A7003E
:101100002708AC002608AB002508AA002408A9007F
:101110002C08C9002B08C8002A08C7002908C600E7
:10112000CD01CC01CB01CA018A1183120D248A158D
:1011300003189C28031DA128F701F801F901FA0101
:10114000292983162C08B0002B08AF002A08AE000E
:101150002908AD00B601AD30B50035088400831311
:10116000361883170008BA01B9007F30B907031891
:10117000BA0A03103A0CFA00390CF900B900350824
:101180008400831336188317390880003008B400B0
:101190002F08B3002E08B2002D08B1002C08C9009A
:1011A0002B08C8002A08C7002908C6003008CD004F
:1011B0002F08CC002E08CB002D08CA008A118312FC
:1011C00042218A15831083163008CD002F08CC00E9
:1011D0002E08CB002D08CA007A08D1007908D0006B
:1011E0007808CF007708CE008A118312C7228A15AB
:1011F0007A088316B0007908AF007808AE00770847
:10120000AD00350884008313361883178003340833
:10121000C9003308C8003208C7003108C6003008CA
:10122000CD002F08CC002E08CB002D08CA008A1153
:1012300083120D248A1503191F298316C6288316C5
:101240003108F7003208F8003308F9003408FA00D2
:1012500083127A08EF007908EE007808ED0077082D
:10126000EC000230EB076F088316CD0083126E0886
:101270008316CC0083126D088316CB0083126C0892
:101280008316CA0083126F088316D10083126E087A
:101290008316D00083126D088316CF0083126C086A
:1012A0008316CE008A1183120E228A157A088316BD
:1012B000A3007908A2007808A1007708A0003730C1
:1012C000CD00BF30CC007D30CB00CA002308D10058
:1012D0002208D0002108CF002008CE008A118312F6
:1012E0000E228A1577088316A4007808A5007908CD
:1012F000A6007A08A70083102708CD002608CC0096
:101300002508CB002408CA003D30D100AA30D00007
:101310009330CF008130CE008A118312C7228A1504
:101320007A08F3007908F2007808F1007708F000F5
:1013300073088316CD007208CC007108CB007008CA
:10134000CA002308D1002208D0002108CF002008BD
:10135000CE008A1183120E228A1577088316A40004
:101360007808A5007908A6007A08A7008310270846
:10137000CD002608CC002508CB002408CA00EE309A
:10138000D1005030D0003330CF008130CE008A11F0
:101390008312C7228A157A08F3007908F2007808C8
:1013A000F1007708F0008316CD01CC01CB017F302E
:1013B000CA002308D1002208D0002108CF0020084D
:1013C000CE008A1183120E228A1577088316A40094
:1013D0007808A5007908A6007A08A70083102708D6
:1013E000CD002608CC002508CB002408CA000A300E
:1013F000D1008D30D000B130CF008130CE008A11C5
:101400008312C7228A157A08FE007908FD00780841
:10141000FC007708FB007E088316CD007D08CC0019
:101420007C08CB007B08CA002308D1002208D0002A
:101430002108CF002008CE008A1183120E228A15BF
:1014400077088316A4007808A5007908A6007A0812
:10145000A70083102708CD002608CC002508CB0064
:101460002408CA00EE30D1005030D0003330CF0015
:101470008130CE008A118312C7228A157A08FE00B5
:101480007908FD007808FC007708FB006F088316D8
:10149000CD0083126E088316CC0083126D0883166C
:1014A000CB0083126C088316CA007308D10072083F
:1014B000D0007108CF007008CE008A1183120E226E
:1014C0008A1577088316A4007808A5007908A60075
:1014D0007A08A700C9002608C8002508C700240804
:1014E000C6007E08CD007D08CC007C08CB007B08C0
:1014F000CA008A11831242218A157A08F3007908FA
:10150000F2007808F1007708F000EB1CB72A831688
:10151000CD01CC01CB018030CA007308D100720824
:10152000D0007108CF007008CE008A1183120E22FD
:101530008A158314DB308316CD000F30CC00493080
:10154000CB007F30CA007A08D1007908D000780833
:10155000CF007708CE008A118312C7228A157A0835
:10156000F3007908F2007808F1007708F000741CA5
:10157000BC2A7108803AF1006B1CDC2A8314DB3032
:101580008316CD000F30CC004930CB007F30CA002D
:101590007308D1007208D0007108CF007008CE0027
:1015A0008A118312C7228A157A08F3007908F2009B
:1015B0007808F1007708F0007008F7007108F8006B
:0A15C0007208F9007308FA00080031
:102000002708D9003C30DA000A121B200A1678088B
:1020100026078316CB01CA000A12831230200A1643
:102020007A08D8007908D7007808D6007708D50054
:102030002408D900DB012508DA005908013A031900
:102040004328033A03194428013A03194928073A57
:1020500003194E28013A03195328033A0319582843
:10206000013A03195D280F3A03196228013A03194E
:102070006728033A03196C28013A03197328073AB1
:1020800003197A288128CD281F30DA070318DB0AC4
:10209000CD283A30DA070318DB0ACD285930DA07A1
:1020A0000318DB0ACD287730DA070318DB0ACD28BE
:1020B0009630DA070318DB0ACD28B430DA070318A4
:1020C000DB0ACD28D330DA070318DB0ACD28F2303B
:1020D000DA070318DB0ACD280630DA0701300318C7
:1020E0000230DB07CD282F30DA0701300318023029
:1020F000DB07CD284D30DA07013003180230DB074B
:10210000CD28043003178D0000308F0083168C1704
:102110000C140000000083120C087F390319CB282F
:102120000313DC0003170D080313DD0003170F086A
:102130000313DE005C08E5000A124F200A165D0852
:1021400003178D0003135E0803178F0083168C1787
:102150000C140000000083120C0D0E0D7F390319C2
:10216000CB280313DC0003170D080313DD0003174E
:102170000F080313DE005C08E5000A124F200A1660
:102180005D0803178D0003135E0803178F008D0A87
:1021900003198F0A86280313CD28073003178D00F3
:1021A00000308F00031005300313DC000A12732087
:1021B0000A16103084005B08DD005A08DC000A12A1
:1021C000C2200A160D30E5000A124F200A160A3006
:1021D000E5000A124F200A165A08F8005B08F900B9
:1021E00079088316CB007808CA000A1283123020BF
:1021F0000A167A08B4007908B3007808B2007708A4
:10220000B1003408DC003308DB003208DA003108A2
:10221000D9003F30E0007E30DF007C30DE007E30D1
:10222000DD009A30EE009930ED003B30EC00833059
:10223000EB000A1285220A167708E1007808E2000E
:102240007908E3007A08E400E6010408E500661076
:10225000831B661483145C088316CD0083125B080D
:102260008316CC0083125A088316CB0083125908B8
:102270008316CA00D101D0012230CF008530CE00B4
:102280000A128312C7220A1665088400831366188F
:10229000831760088316CD0083125F088316CC0075
:1022A00083125E088316CB0083125D088316CA0072
:1022B0007A08D1007908D0007808CF007708CE00DE
:1022C0000A1283120E220A167708E7007808E8003F
:1022D0007908E9007A08EA00EE007908ED0078084C
:1022E000EC007708EB000A1285220A167708E7004F
:1022F0007808E8007908E9007A08EA00EE00790831
:10230000ED007808EC007708EB000A1244260A1664
:1023100064088316CD00831263088316CC008312F1
:1023200062088316CB00831261088316CA007A08FC
:10233000D1007908D0007808CF007708CE000A12C3
:1023400083120E220A167A08DC007908DB0078086E
:10235000DA007708D9005908F7005A08F8005B0836
:10236000F9005C08FA007A08C0007908BF00780814
:10237000BE007708BD002808D900EE01ED017030DD
:10238000EC008230EB000A1285220A167708DE0084
:102390007808DF007908E0007A08E1008316CB01B5
:1023A000831259088316CA000A12831230200A16B3
:1023B00061088316CD00831260088316CC00831257
:1023C0005F088316CB0083125E088316CA007A0862
:1023D000D1007908D0007808CF007708CE000A1223
:1023E00083120E220A167A08DD007908DC007808CC
:1023F000DB007708DA005A08F7005B08F8005C0891
:10240000F9005D08FA007A08C4007908C30078086A
:10241000C2007708C1003408DC003308DB00320852
:10242000DA003108D90083145C088316CD008312CA
:102430005B088316CC0083125A088316CB008312E4
:1024400059088316CA00D101D0012230CF0085304F
:10245000CE000A128312C7220A163F308316CD001F
:102460007E30CC007C30CB007E30CA007A08D100B0
:102470007908D0007808CF007708CE000A128312BE
:102480000E220A167708E1007808E2007908E300D6
:102490007A08E400EE007908ED007808EC0077088F
:1024A000EB000A1285220A167A08E0007908DF009C
:1024B0007808DE007708DD008316CD01CC01CB0162
:1024C0008030CA00831260088316D10083125F082F
:1024D0008316D00083125E088316CF0083125D0836
:1024E0008316CE000A1283120E220A167708E10024
:1024F0007808E2007908E3007A08E400EE00790841
:10250000ED007808EC007708EB000A1244260A1662
:1025100085308316CD00EB30CC001D30CB008230EF
:10252000CA007A08D1007908D0007808CF0077086F
:10253000CE000A1283120E220A167708E1007808EC
:10254000E2007908E3007A08E4006008F6005F081A
:10255000F5005E08F4005D08F3000A126F240A1605
:10256000C3308316CD00F530CC007030CB00813005
:10257000CA007A08D1007908D0007808CF0077081F
:10258000CE000A1283120E220A16E6010408E500A4
:102590006610831B6614831464088316CD008312AF
:1025A00063088316CC00831262088316CB00831263
:1025B00061088316CA007A08D1007908D00078082B
:1025C000CF007708CE000A128312C7220A166508C8
:1025D00084008313661883177708E1007808E20007
:1025E0007908E3007A08E4006008EE005F08ED0077
:1025F0005E08EC005D08EB000A1244260A168316FA
:10260000CD01CC014030CB007F30CA007A08D10028
:102610007908D0007808CF007708CE000A1283121C
:102620000E220A16E8010408E7006810831B6814EC
:10263000831464088316CD00831263088316CC00CC
:10264000831262088316CB00831261088316CA00C6
:102650007A08D1007908D0007808CF007708CE003A
:102660000A128312C7220A166708840083136818A7
:1026700083177A08E0007908DF007808DE00770821
:10268000DD005D08F7005E08F8005F08F9006008EB
:10269000FA007A08C8007908C7007808C6007708E9
:1026A000C50030088316C90083122F088316C8009E
:1026B00083122E088316C70083122D088316C600C6
:1026C0000A1283124E240A167808D9005908DA0033
:1026D0004408DE004308DD004208DC004108DB005E
:1026E0004808E2004708E1004608E0004508DF002E
:1026F0008316CB0183125A088316CA000A1283126A
:1027000030200A1683147A088316CD007908CC008D
:102710007808CB007708CA0083125E088316D100C0
:1027200083125D088316D00083125C088316CF00E5
:1027300083125B088316CE000A128312C7220A1680
:102740008316CD01CC01CB018130CA007A08D100BB
:102750007908D0007808CF007708CE000A128312DB
:102760000E220A167708E7007808E8007908E900E1
:102770007A08EA0083107A088316CD00831279085C
:102780008316CC00831278088316CB008312770857
:102790008316CA00831262088316D100831261086F
:1027A0008316D000831260088316CF0083125F085F
:1027B0008316CE000A128312C7220A167A08E60090
:1027C0007908E5007808E4007708E3006308F7007B
:1027D0006408F8006508F9006608FA007A08CC0079
:1027E0007908CB007808CA007708C9005808DC00CF
:1027F0005708DB005608DA005508D9004C08E000FD
:102800004B08DF004A08DE004908DD006008831637
:10281000C90083125F088316C80083125E088316FE
:10282000C70083125D088316C600CD01CC0170304D
:10283000CB008430CA000A12831242210A16831088
:102840005C088316CD0083125B088316CC008312CC
:102850005A088316CB00831259088316CA007A08D7
:10286000D1007908D0007808CF007708CE000A128E
:102870008312C7220A167A08E4007908E300780870
:10288000E2007708E1006108F7006208F8006308D9
:10289000F9006408FA007A08D0007908CF007808B7
:1028A000CE007708CD005008DC004F08DB004E0852
:1028B000DA004D08D900EE01ED017030EC008230F5
:1028C000EB000A1285220A167708DD007808DE0080
:1028D0007908DF007A08E000E2010408E1006210F4
:1028E000831B621483145C088316CD0083125B087B
:1028F0008316CC0083125A088316CB008312590822
:102900008316CA00D101D0014030CF008230CE0002
:102910000A128312C7220A16610884008313621800
:10292000831760088316CD0083125F088316CC00DE
:1029300083125E088316CB0083125D088316CA00DB
:102940007A08D1007908D0007808CF007708CE0047
:102950000A1283120E220A167A08DC007908DB00BC
:102960007808DA007708D9005908F7005A08F80003
:102970005B08F9005C08FA007A08D4007908D300F3
:102980007808D2007708D1002C08EE002B08ED0063
:102990002A08EC002908EB000A1285220A167A0898
:1029A000AC007908AB007808AA007708A9004008B5
:1029B000EE003F08ED003E08EC003D08EB000A1277
:1029C00044260A167708D9007808DA007908DB006F
:1029D0007A08DC002C08EE002B08ED002A08EC0039
:1029E0002908EB000A1244260A165C088316CD005B
:1029F00083125B088316CC0083125A088316CB001F
:102A0000831259088316CA007A08D1007908D000C9
:102A10007808CF007708CE000A1283120E220A1619
:102A20007708D9007808DA007908DB007A08DC003A
:102A30004008F6003F08F5003E08F4003D08F300AA
:102A40000A126F240A167708DD007808DE0079087C
:102A5000DF007A08E0002C08F6002B08F5002A08B1
:102A6000F4002908F3000A126F240A16600883167E
:102A7000CD0083125F088316CC0083125E08831694
:102A8000CB0083125D088316CA007A08D10079084A
:102A9000D0007808CF007708CE000A1283120E22E9
:102AA0000A167708DD007808DE007908DF007A086A
:102AB000E0005408F6005308F5005208F4005108ED
:102AC000F3000A126F240A1660088316CD008312E1
:102AD0005F088316CC0083125E088316CB00831236
:102AE0005D088316CA007A08D1007908D0007808FA
:102AF000CF007708CE000A1283120E220A16DE01DA
:102B00000408DD005E10831B5E1483105C088316CE
:102B1000CD0083125B088316CC0083125A088316FB
:102B2000CB00831259088316CA007A08D1007908AD
:102B3000D0007808CF007708CE000A128312C7228F
:102B40000A165D08840083135E1883177708D9007E
:102B50007808DA007908DB007A08DC005C08E2001B
:102B60005B08E1005A08E0005908DF006208EA004B
:102B70006108E9006008E8005F08E700EB010A125D
:102B80008A1500200A168A117A08E6007908E500FD
:102B90007808E4007708E3006308F7006408F800A9
:102BA0006508F9006608FA007A08B8007908B700E5
:102BB0007808B6007708B5004008EE003F08ED0041
:102BC0003E08EC003D08EB000A1244260A1677087E
:102BD000D9007808DA007908DB007A08DC002C08D4
:102BE000F6002B08F5002A08F4002908F3000A1261
:102BF0006F240A165C088316CD0083125B088316C7
:102C0000CC0083125A088316CB008312590883160E
:102C1000CA007A08D1007908D0007808CF00770878
:102C2000CE000A1283120E220A167708D9007808FD
:102C3000DA007908DB007A08DC004008F6003F087B
:102C4000F5003E08F4003D08F3000A126F240A164E
:102C50007708DD007808DE007908DF007A08E000F8
:102C60002C08EE002B08ED002A08EC002908EB00E8
:102C70000A1244260A1660088316CD0083125F08E4
:102C80008316CC0083125E088316CB0083125D0886
:102C90008316CA007A08D1007908D0007808CF00DE
:102CA0007708CE000A1283120E220A167708DD007A
:102CB0007808DE007908DF007A08E0005408F600A2
:102CC0005308F5005208F4005108F3000A126F246B
:102CD0000A1660088316CD0083125F088316CC00A5
:102CE00083125E088316CB0083125D088316CA0028
:102CF0007A08D1007908D0007808CF007708CE0094
:102D00000A1283120E220A16DE010408DD005E108C
:102D1000831B5E1483145C088316CD0083125B084A
:102D20008316CC0083125A088316CB0083125908ED
:102D30008316CA007A08D1007908D0007808CF003D
:102D40007708CE000A128312C7220A165D08840093
:102D500083135E1883177708D9007808DA0079089A
:102D6000DB007A08DC003808F6003708F500360882
:102D7000F4003508F3000A126F240A165C08831663
:102D8000C90083125B088316C80083125A08831691
:102D9000C700831259088316C6007A08CD00790847
:102DA000CC007808CB007708CA000A1283124221AF
:102DB0000A167708D9007808DA007908DB007A0863
:102DC000DC005C08E2005B08E1005A08E0005908FA
:102DD000DF006208EA006108E9006008E8005F08B7
:102DE000E7000130EB000A128A1500200A168A114A
:102DF0007A08E6007908E5007808E4007708E3003F
:102E00006308F7006408F8006508F9006608FA002E
:102E10007A08BC007908BB007808BA007708B900C6
:102E20003808DC003708DB003608DA003508D9003E
:102E30000A126F260A167808A3003C08DC003B083B
:102E4000DB003A08DA003908D9000A126F260A16A0
:102E5000FA017808A1007A08A2008316C901C80106
:102E6000C701C601831254088316CD00831253088C
:102E70008316CC00831252088316CB0083125108AC
:102E80008316CA000A1283120D240A16031C532F3C
:102E90002108683CA1002208031C220F512F013099
:0C2EA000522F013CA2008A110A12B02F30
:04400E00F52CFF3F4F
:00000001FF
